:020000040000FA
:040000004CEF06F0CB
:08000800056ED8CF06F0E0CF31
:1000100007F00001E9CF0DF0EACF08F0E1CF09F0D9
:10002000E2CF0AF0D9CF0BF0DACF0CF0F3CF14F017
:10003000F4CF15F0FACF16F000C00FF001C010F0A9
:1000400002C011F003C012F004C013F09DAA2CEFFF
:1000500000F09EBADCEF00F00FC000F010C001F01D
:1000600011C002F012C003F013C004F00DC0E9FF8C
:1000700008C0EAFF088E09C0E1FF0AC0E2FF0BC01A
:10008000D9FF0CC0DAFF14C0F3FF15C0F4FF16C08F
:10009000FAFF055007C0E0FF06C0D8FF1000F2CFFE
:1000A0000EF0F29EF76AB80FF66E000EF722090006
:1000B000F5500EBEF28E120021303036302530322F
:1000C000580D0A00F2CF0EF0F29EF76ADE0FF66EC0
:1000D000000EF7220900F5500EBEF28E12002130FC
:1000E00030373130310D0A00F2CF0EF0F29EF76A50
:1000F000020FF66E010EF7220900F5500EBEF28EC9
:100100001200213030373130300D0A00F2CF0EF0BE
:10011000F29EF76A260FF66E010EF7220900F550DF
:100120000EBEF28E120021303038302530344C555E
:100130000D0A0000F2CF0EF0F29EF76A4E0FF66E37
:10014000010EF7220900F5500EBEF28E120021308A
:100150003038312530364C550D0A0000F2CF0EF004
:10016000F29EF76A760FF66E010EF7220900F5503F
:100170000EBEF28E120021303038322C253032582B
:100180002C253032582C2530364C5500F2CF0EF04D
:10019000F29EF76AA60FF66E010EF7220900F550DF
:1001A0000EBEF28E120021303066300D0A000400BF
:1001B0009EA8FDD7AD6E000C04009EAAFDD7AECF61
:1001C00084F019B673D019B809D08451240805E118
:1001D0001988199A240E326E316A68D08451240A23
:1001E00003E0290A06E033D0199A240E326E316AF0
:1001F0005DD0199831522AE033501C5C27E119BABE
:1002000002D0312C04D0198E660E316E1FD019BC6D
:1002100005D0020E315C1C6E198618D02F50325C4E
:10022000D8803054326E010E315C036A1C0FE96EC7
:10023000000E0320EA6EEF50325C05E1030E315CE4
:100240001C6E198603D0198E630E316E2FD0845127
:10025000322619BA04D0198A84C02FF027D0199AEF
:1002600084C030F02FC084F0843BF00E84172FAC94
:1002700002D0900E842730500F0B842730AC02D070
:10028000090E8427036A31501C0FE96E000E03200B
:10029000EA6E84C0EFFF312A3150120807E2199844
:1002A00033501C5C03E1198E6F0E316E19A631D0EC
:1002B0001D5007E0010A0EE0030A17E0050A1FE0DF
:1002C00028D0198E1C5203E1300E316E02D0660E1A
:1002D000316E1FD0198E1C2C05D01EC033F0610E5C
:1002E000316E02D0660E316E14D0198E1C5204E1AC
:1002F000197C610E316E02D0660E316E0AD0198EF5
:100300001C5204E13480610E316E02D0660E316EF3
:1003100000D019AE6ED0199E210E49DF33C084F093
:10032000843B84510F0B300F846F8451390802E2F3
:10033000070E8427210E8425326E845138DF335016
:100340000F0B300F846F8451390802E2070E8427A7
:1003500084512DDF8451322619A620D01996300EF3
:1003600026DF300E1D24856F22DF300E32241D243F
:10037000300F326E1D5212E11C5210E1300E17DFA9
:10038000310E15DF390E13DF330E11DF300E0FDFA4
:10039000300E0DDF300E0BDF5D0E3226315007DFE1
:1003A0003150322619AC19D032C084F0843B8451CC
:1003B0000F0B300F846F8451390802E2070E842737
:1003C0008451F5DE32500F0B300F846F84513908A1
:1003D00002E2070E84278451EADE0D0EE8DE0A0EE3
:1003E000E6DE34A006D0000EE2DE000EE0DE349041
:1003F000FF00000E9EBA010E0108D8B4DDD69E9A09
:100400002CEF00F0386A385013080AE3036A3850BA
:100410001C0FE96E000E0320EA6EEF6A382AF3D74C
:10042000316A37C032F036C033F019961998199AEC
:10043000199C199E34906AEF06F0700ED36E400E30
:100440009B6ED350D00E896E8A6AC00E8B6EC90E19
:10045000926E200E936E800E946E3492C150C00B3B
:100460001E09C16EC050C00B3F09C06EC08EC28055
:10047000C69A010EC66E000EC76ED190800ED56E64
:10048000CD6A000ECA6E000ECB6E070EB46E92508F
:10049000926E04001A0E006E002EFED7B450A19C7E
:1004A000B56A9D8AC00EF2126CEF06F0EA6A710E10
:1004B000E96EEF5011E00A0E016EBF0E006E0400EF
:1004C000002EFDD7012EF9D75E0E006E002EFED74E
:1004D00000D00400EF2EEFD7000C8B50F00B696EAC
:1004E00068500F0B69108B6E82500F0B696E69C0DC
:1004F00001F0000C69BE11D00F0E006E68380016B6
:100500000A0E005C03E2300E002602D0695000267D
:10051000005004009EA8FDD7AD6E0F0E68160A0E9F
:10052000685C02E2300E02D0699E6950682668500D
:1005300004009EA8FDD7AD6E000C020E6B5E0BE3AF
:10054000EA6A6B0EE96EEF5006E003D000D000D0EF
:100550000400EF2EFBD7C9EF02F067500F0801E24D
:10056000676A000E016EC250C30B0110C26E675065
:10057000070B686EF80E8A1668508A128A868A8877
:1005800067A602D08A9801D08A960400C70E6B6EC7
:10059000D4D7C282C2B2FED7C3CF69F0C4CF6AF04B
:1005A00069C001F06AC002F002EF05F0EACF70F016
:1005B000E9CF6FF06938F0096B6E6B26E20F6C6E55
:1005C000320F6E6E69500F0B6C266C266E26E90F8B
:1005D0006D6E6D266D2668380F0B6D266E266D3696
:1005E0006E366E1E6E3668500F0B6E266B36070E1B
:1005F0006A6E0A0E6D066E26FDE36C066D26FDE33F
:100600006B066C26FDE36A066B26FDE3EA6A6A0E5A
:10061000E96E070E6F146F9CE9266E0EE95CD8B484
:100620006F8CEF50006E08E16FBC06D06FB80DD034
:100630006FB602D0200E03D06F866F98300E002662
:10064000005004009EA8FDD7AD6EEE506FACE5D70C
:1006500017EF05F07D6A7E6A010E7F6EDA6AD96A4D
:10066000826B750E816FEA6A790EE96E82C0E2FFD5
:1006700081C0E1FF7FC080F0D890E550EE02F350DA
:100680007D22F4507E22802FF7D77DC0DEFF7EC012
:100690007DF07E6AD8B07E2A812BD8B4822B7F2A47
:1006A0007F500508E0E1000C69500F0801E2696A1B
:1006B000000E016EC250C30B0110C26E6950070BD1
:1006C0006A6EF80E8A166A508A128A868A8869A625
:1006D00002D08A9801D08A96020E716EE7DEC2823D
:1006E000C2B2FED7C3CF6BF0C4CF6CF069500A081A
:1006F0001CE3746A736A6CC072F06BC071F074C0F2
:1007000078F073C077F06CC076F06BC075F07C6ADF
:100710007B6A7B0E7A6E4A0E796E9CDF01C06DF0AB
:1007200002C06EF003C06FF0706A69500B081CE1E4
:10073000746A736A6CC072F06BC071F074C078F048
:1007400073C077F06CC076F06BC075F07C6A7B6A22
:10075000070E7A6EF40E796E7DDF01C06DF002C077
:100760006EF003C06FF0706A69500B0804E2706AA3
:100770006F6A6E6A6D6A6DC000F06EC001F06FC086
:1007800002F070C003F0000C006A016A026A036A9A
:100790007F6A806B816B826B7E507D107C107B103A
:1007A0002CE0200E836FD8907736783679367A36FB
:1007B0007F368037813782377E50825D08E17D50F9
:1007C000815D05E17C50805D02E17B507F5C0FE341
:1007D0007B507F5E7C50D8A07C3C805F7D50D8A051
:1007E0007D3C815F7E50D8A07E3C825FD880003601
:1007F000013602360336832FD6D7EA6A7F0EE96EBA
:10080000000CE9506F6E3B0E766E9A0E756ECA0E36
:10081000746E736A0A0E716E6EC07AF06DC079F0F4
:100820006CC078F06BC077F076C07EF075C07DF05C
:1008300074C07CF073C07BF0A7DF0150EFCF6BF08A
:10084000ECCF6CF0ECCF6DF0ECCF6EF000520FE11E
:100850007150010A0CE06F500BE00F0B715C01E06E
:100860000EE26FBE0CD06FBC03D0200E02D06F6AB8
:10087000300E0026005004009EA8FDD7AD6E76C055
:100880007AF075C079F074C078F073C077F07E6A42
:100890007D6A7C6A0A0E7B6E77DF03C076F002C049
:1008A00075F001C074F000C073F0712EB5D7000C64
:1008B0006750F00B6B6E6B3A300E6B266B5039083D
:1008C00002E2070E6B2669C0E9FF6AC0EAFF6BC04F
:1008D000EFFF67500F0B6C6E6D6A300E6C246B6E01
:1008E0006B50390802E2070E6B26010E6924E96E8F
:1008F000000E6A20EA6E6BC0EFFF000CABA202D0C4
:10090000AB98AB8819A6B2D11D50600A0EE0100A50
:1009100044E0010A54E0F10AD8B46FD0010AD8B417
:1009200091D0030AD8B4BBD075D11C2C33D01EA8EB
:100930000FD03F0E92161EAA08D0899834B204D068
:10094000C80E716EB3DD348202D08988349207D02C
:1009500089883492C80E716EA9DDC00E92121E50A5
:100960000F0B676E686EB9DD01C036F0676A6750BD
:100970004FEC00F0672A1BDC050E675CF8E136C01F
:1009800068F0370E696EB6DD0D0E11DC0A0E0FDC55
:100990001C6A02D0660E1C6E40D11C2C0DD01EA00D
:1009A00002D08B8A01D08B9A1EA202D08B8801D0F4
:1009B0008B98610E1C6E02D0660E1C6E2ED11C52DE
:1009C00019E181AA0BD0676A675062EC00F0672AD0
:1009D000D7EC00F0090E675CF7E10AD0676A675050
:1009E00074EC00F0672AD7EC00F0090E675CF7E1C1
:1009F0001C6A02D0660E1C6E10D11C2C20D01EC0AA
:100A000067F0ABD502C038F001C037F0676A6750B5
:100A100086EC00F0672AD7EC00F0050E675CF7E182
:100A2000090EE96E38C069F037C068F0BFD50D0E09
:100A3000D7EC00F00A0ED7EC00F01C6A02D0660E6C
:100A40001C6EEBD01C2C28D01EC069F02DDE03C01C
:100A50003CF002C03BF001C03AF000C039F0676AD8
:100A600067509AEC00F0672AD7EC00F0050E675C3F
:100A7000F7E1460EE96E3CC06EF03BC06DF03AC047
:100A80006CF039C06BF0BDDE0D0ED7EC00F00A0E35
:100A9000D7EC00F01C6A02D0660E1C6EBED01C2C77
:100AA000B6D01EA80FD03F0E92161EAA08D0899865
:100AB00034B204D0C80E716EF9DC348202D0898859
:100AC000349207D089883492C80E716EEFDCC00E64
:100AD00092121E500F0B676E686EFFDC01C03DF076
:100AE0000B0E696EE1DD03C041F002C040F001C0B1
:100AF0003FF000C03EF0676A6750AEEC00F0672A36
:100B0000D7EC00F0060E675CF7E11EC068F0370E08
:100B1000696EF0DC2C0ED7EC00F03DC068F0370EAB
:100B2000696EE8DC2C0ED7EC00F0460EE96E41C091
:100B30006EF040C06DF03FC06CF03EC06BF061DE07
:100B4000666A665009081DE36650040DF350036A97
:100B50003E0F016E000E032201C067F003C068F073
:100B600066C069F0A1DD68C0EAFF67C0E9FF00C0A8
:100B7000EFFF01C0ECFF02C0ECFF03C0ECFF662AF0
:100B8000E0D7666A6650090821E36650040DF35009
:100B9000036A3E0FE96E000E0320EA6EEFCF67F0A6
:100BA000ECCF68F0ECCF69F0ECCF6AF02C0ED7EC0C
:100BB00000F0460EE96E6AC06EF069C06DF068C064
:100BC0006CF067C06BF01DDE662ADCD70A0E696E1A
:100BD0006BDD03C041F002C040F001C03FF000C037
:100BE0003EF02C0ED7EC00F0460EE96E41C06EF0E0
:100BF00040C06DF03FC06CF03EC06BF002DE0D0EE9
:100C0000D7EC00F00A0ED7EC00F01C6A02D0660E9A
:100C10001C6E03D03F0E1C6E00D01C5226E0210E2D
:100C2000D7EC00F0686A33C067F06A6A2F0E696E0D
:100C30003FDE2F50D7EC00F03050D7EC00F0686A60
:100C40001DC067F06A6A2F0E696E32DE2F50D7EC36
:100C500000F03050D7EC00F01C50D7EC00F00D0E37
:100C6000D7EC00F00A0ED7EC00F019966EEF06F004
:100C70001A2AD8B41B2A1A3C0CD01B507F0809E151
:100C800019801972899A19B2898A19841B6A1A6A99
:100C900001D019906FEF06F0F86AD09E088EEA6ACC
:100CA000E96AB886440EAF6E000EB06EA60EAC6E4A
:100CB000900EAB6EC150C00B0F09C16E070EB46E23
:100CC0001990199219941A6A1B6A3590366A376A14
:100CD00002EF02F01DEF02F0040010D6C9D781BA6E
:100CE0001AD08B988B9A640E716E56EC02F081BA12
:100CF00002D00400FCD78B888B8A640E716E56EC90
:100D000002F0366A3650C6EC00F0362AD7EC00F016
:0A0D1000070E365CF7E1E0D70300A0
:020000040030CA
:0E0000000048160F000181000FC00FE00F40F6
:00000001FF
